:0200000035C009
:02000400F0C04A
:10002000440054004D004600200044006500630079
:100030006F006400650072002000620079002000FB
:1000400000007700770077002E0069006E006600E0
:1000500069006400690067006D002E006E00650095
:100060007400000045006E006400000000E007BB63
:1000700000E701BB94980FED0DBF06E109B908E058
:100080000AB90CE205BF00E80BBF00EC0ABF1AD0AA
:1000900024D053D097D074D069D050E4A0E6B0E01B
:1000A00001E0C02EA22E622F00E8600F78948099A4
:1000B00003C0809BFECF1DD18299F9CF829BFECFDA
:1000C00041D1F5CF01E022D002E020D008E31ED0DC
:1000D0000CE01CD006E01AD00895F0E0E0E2C895EC
:1000E000002D003021F010D0E395E395F8CF00EC1F
:1000F0000DD0F0E0E2E4C895002D003021F004D0EE
:10010000E395E395F8CF0895959A01C095981FEF70
:1001100017BB08BB0CD0969A0AD0969800E107D07E
:100120000A950030E1F700E007BB08BB089513EB28
:1001300000001A951030E1F7089518D0F0E0E0E2E1
:10014000C895002D003029F00CB932D0E395E39525
:10015000F7CFF0E0E2E4C895002D003029F00CB9AB
:1001600027D0E395E395F7CF01D008950AE00CB9C5
:100170001FD00AE00CB91CD00DE00CB919D00895BD
:10018000122F13951EBBE09A0DB3069506950695A2
:10019000069512D00CB90CD00DB30F700DD00CB960
:1001A00007D00FE7020F101710F41395EBCF089547
:1001B0005E9BFECF5E9A08950E3011F400270895DD
:1001C0000063089522272EBBE09A31E00DB3007F33
:1001D000003F09F4089533270DB30F700F3009F471
:1001E00008952395F0CFF89400E007BB949A00009F
:1001F00046B394984F704A3009F4442700E3400F07
:10020000503510F011D004C00C2D013009F442D04B
:100210004D93042F79DF53954CB9CADF13D06A2D63
:1002200000E8600F7894189501E070DFA0E60D916A
:100230006BDFA037E0F3A0E650E4A22E00EC66DF0F
:10024000CC2408954F70303081F42EBBE09A0DB36A
:10025000007F042B0DBB11D023952EBBE09A0DB36C
:10026000006F0DBB0AD031E00895042F02950F6096
:100270002EBB0DBB02D03327089504E00CBBE19ADE
:100280000FEF003021F00A9500000000FACFE1994D
:10029000FECF0895AF9201E039DFBB2408E0A01A39
:1002A000AEBAE09A313059F4AEBAE09A0DB3069581
:1002B00006950695069510E3010F26DFB3940DB35E
:1002C0000F7010E3010F20DFB394A3940B2D0031C6
:1002D00058F3AF9000EC1ADFA0E60A2F0052051782
:1002E00019F00D9111DFF9CF00E8050F0FDFCC24D5
:1002F00008950A2D10E8010F162F101708F0089521
:1003000001E004DF762F45D000EC00DF0A2D18E76E
:10031000010F162F101768F0A0E60A2F00520517DC
:1003200019F00D91F1DEF9CF00E8050FEFDECC24D6
:1003300006C0762F08E0700F2CD001E0C02E08E038
:10034000600F08950A2D11E0010F162F101708F401
:10035000089501E0DBDE0A2D19E0010F162F1017BA
:1003600050F4F0E0E4E6C895002D003041F0CCDE1A
:10037000E395E395F8CF762F00E1701B0AD000ECEF
:10038000C5DE762F08E0701B04D001E0C02E685057
:100390000895BB247EBBE09A313059F47EBBE09ACD
:1003A0000DB3069506950695069510E3010FACDE94
:1003B000B3940DB30F7010E3010FA6DEB3947395E1
:0803C0000B2D003158F30895E4
:00000001FF
